:040000006F00204429
:100004000000000000000000480200004A02000056
:100014000000000040040000000000000000000098
:100024004004000040040000000000000000000044
:100034003C1E00000000000040040000000000001E
:10004400400400004004000040040000400400009C
:10005400400400004004000040040000400400008C
:10006400701900004004000040040000BE160000A7
:10007400400400004004000040040000400400006C
:10008400400400004004000040040000400400005C
:10009400400400004004000040040000400400004C
:1000A400400400004A1E0000400400004004000018
:1000B400201E0000721D00004004000040040000E7
:1000C400400400004004000040040000400400001C
:1000D400400400004004000040040000E61C00004E
:1000E400081A00004004000040040000400400001E
:1000F400400400002C1D00004004000040040000E7
:1001040040040000400400004004000040040000DB
:100114004004000000000000000000000000000097
:1001240000000000000000000000000000000000CB
:0C013400000000000000000000000000BF
:10014000397101436EC619A0397141536AC866CA34
:1001500062CC5ECE19A0397101535AD056D252D416
:100160004ED64AD826DA22DC06DE3301614082828E
:1001700041114AC026C222C406C68282B24D410144
:10018000024D924C224CB24B4101024B924A224A00
:10019000B2494101024992442244B2404101828065
:1001A0003D432A876373C3029377F700BDEFADE544
:1001B000937606FF3D8ABA960CC34CC30CC74CC756
:1001C0004107E36BD7FE11E28280B306C3408A0683
:1001D0009702000096966780A6002307B700A30643
:1001E000B7002306B700A305B7002305B700A30493
:1001F000B7002304B700A303B7002303B700A3028B
:10020000B7002302B700A301B7002301B700A30082
:10021000B7002300B700828093F5F50F9396850011
:10022000D58D93960501D58D61B7939627009702DA
:10023000000096968682E78086FA9680C1171D8F09
:100240003E96E374C3F8A5B701A001A0EFF25FF2F8
:100250000545EF0050399922EF1070517165130573
:100260000520EF10D052B707002083A5071037559F
:1002700000001305054FEF40E00AED23AA8537552E
:10028000000013050550EF40E009EF20A03FEF20EC
:10029000603B014501B7EFF2BFED371402401C404F
:1002A0003707FF08411193E717001CC05C40F98F26
:1002B0005CC01C403707F7FE6D17F98F1CC01C404F
:1002C0003707FCFF7D17F98F1CC05C40370701FF23
:1002D0007D17F98F5CC0B7079F001CC4EF00B017F3
:1002E00002C402C6B7270240054798C31C404167B5
:1002F000B7160240D98F1CC03706020005679C4222
:10030000F18F3EC6A24785073EC4B24781E7A247A8
:10031000E397E7FEB71702409C431397E700635744
:10032000070685473EC6324785476313F706B7176A
:100330000240D843B706C1FFFD16D8C3D843D8C37F
:10034000D84313670740D8C3D843758FD8C3D84361
:10035000B7061100558FD8C39843B7060001558FD3
:1003600098C3984393166700E3DD06FED843B7169B
:100370000240719BD8C3D84313672700D8C32147D5
:10038000DC42B18BE39EE7FE410129B502C661BFA5
:10039000372702401C43F19B1CC3FDB7B716024030
:1003A000DC42370700201146B18B13070710638F1B
:1003B000C70221466381C70495EB9C42918B9DC780
:1003C000B7470F00938707241CC3B7170240DC43CD
:1003D000918393F6F700B707002093870700B6973D
:1003E00094231C43B3D7D7001CC38280B7177A006D
:1003F00093870720D1BFDC42D4424166C983BD8BBD
:10040000F18E890745466393C700C94781EEB74619
:10041000024083A60680C18A89CEB7167A009386E9
:10042000062021A8B7160240D4421396E600E356F0
:1004300006FEB7163D0093860690B387D70269B7CC
:1004400001A0970100209381E14B17510020130177
:1004500061BB175500001305655C97050020938567
:1004600065BA1386818163FAC5008322050023A043
:10047000550011059105E3EAC5FE13858181938539
:1004800081AE6377B500232005001105E36DB5FE4D
:10049000FD42739002BC8D427390428093028008AB
:1004A0007390023097020000938202B693E232000A
:1004B00073905230EFF03FDE97020000938242D9F2
:1004C0007390123473002030B727014093870740A0
:1004D000631FF500EFF2DFC9854513050020EF002B
:1004E000702A814513050020EF00D02965B1828074
:1004F0005C413707F1E01307F7EF944D7D8F9C4186
:10050000D58FD44DD58FD441A206D58FD98F5CC15C
:100510001C4537F7F1FF1307D77FD4457D8F9C49E2
:10052000D58F94458606D58FD98F1CC55C55370766
:1005300010FF7D177D8FDC29FD1793F7F70FD2078A
:10054000D98F5CD582801C4589C593E717001CC5EF
:100550008280F99BEDBF1C4589C593E707101CC538
:10056000828093F7F7EFE5BF1C4593E787001CC532
:10057000828008450D81058982801C4593E74700EC
:100580001CC582800845098105898280A54763F7DB
:10059000B7048D47138765FF3307F7020328C500AB
:1005A0009D47B397E70093C7F7FFB3F70701B396EB
:1005B000E600DD8E54C5994763E3C70495477D1671
:1005C0003306F6025859FD47B397C70093C7F7FFA4
:1005D000F98F3396C5005D8E50D982800D473387E1
:1005E000E502032805019D47B397E70093C7F7FF8E
:1005F000B3F70701B396E600DD8E14C96DBFB147AE
:1006000063E2C702954765163306F6021859FD479F
:10061000B397C70093C7F7FFF98F3396C5005D8E78
:1006200010D9828095474D163306F6025855FD477E
:10063000B397C70093C7F7FFF98FB395C500DD8D5A
:100640004CD582805C4191C537070004D98F5CC1CD
:100650008280370700FC7D17F98FD5BF3C4989C5DB
:1006600093E707083CC9828093F7F7F7E5BF3C4959
:1006700089C593E707043CC9828093F7F7FBE5BF80
:100680003C4993F7F7FD3CC93C49DD8D2CC982807C
:10069000EFF21FAEB7066745B727024093863612C2
:1006A0003797EFCDD4C31307B79AD8C3D4D301116A
:1006B00098C7D45B1387470313962600E34B06FEC7
:1006C000D457372501401305054093E60620D4D7BB
:1006D000DC5BB7060020D58F1CC31C431C453707C5
:1006E0000E00D98F1CC51C4593E717001CC53C495B
:1006F00093E707043CC91C4593E787001CC52A847F
:100700002285853D75FD37250140832785401305EA
:10071000054093E747001CC52A842285A53575FD51
:10072000372501400546C945814613050540B93DB9
:1007300025462304010037270140B70550001C84DB
:10074000637FF60423040100A54621461C8463FF51
:10075000F606231501002304010095461C8463F16D
:10076000F60E38853C8599460D46B3F7D7020565E8
:10077000130505803357D702B3D7C702BA97C2070C
:10078000C1837C85B727014003A78740799B23A4B9
:10079000E7403C8505611D8D42054185E5BA83270B
:1007A0008740CD8F2324F74083270740898BEDDFD7
:1007B0001C848326C74408108607AA972396D7FE71
:1007C0001C84850793F7F70F5C8495BFA304010091
:1007D0009C846378F6001C84850793F7F70F5C848C
:1007E000B5B798849C840C100607850786072E975A
:1007F000AE970357C7FE83D7C7FE63FDE7029C840D
:100800008607AE9783D7C7FE7C859C84988485072E
:100810008607AE9783D5C7FE931717001810BA97AF
:100820002396B7FE9C8438850C1085078607AE9703
:100830002396E7FE9C84850793F7F70FDC8449BF76
:100840001C841010388589078607B29783D7C7FEA6
:10085000BA97C207C1837C851C84850793F7F70F7D
:100860005C84EDBD03A5C18182801C41416779177D
:10087000F98F1CC123200500232205002324050035
:10088000B707024023260500138787006317E5009A
:10089000D8431367F700D8C382801387C701631654
:1008A000E500D8431367070FFDB7138707036318E5
:1008B000E500D8438566938606F0558FE9BF138718
:1008C00047046315E500D843BD66C5BF1387870598
:1008D0006316E500D843B7060F00C5B71387C706F0
:1008E0006316E500D843B706F000C1BF13870708B9
:1008F0006316E500D843B706000FC1B71387470951
:10090000E31CE5F8D843B70600F045BF1C4161770A
:100910003D0794517D8F9C45D58F9449D58FD449FF
:10092000D58F944DD58FD44DD58FD451D58F945527
:10093000D58FD98F1CC1DC455CC19C411CC5DC41F5
:100940005CC582801C4189C593E717001CC1828069
:1009500041677917F98FDDBF1C4101C6DD8D0CC1E0
:10096000828093C5F5FFFD8DDDBFB70702409C4334
:100970007D8D3335A0008280EFF28FFFFD376FF061
:100980007F81B7070240C8C3828058410328050011
:100990004C4537060140930706403E979346F8FFC3
:1009A000B1C583250640F58D2320B640D043F18E96
:1009B000D4C31443B3E6060114C3184190479346C9
:1009C000F7FF758E90C7D047F18ED4C714454146C6
:1009D0006399C6009447D98E94C7D447558FD8C71A
:1009E0008280B6979443558F98C382801C43F58FBD
:1009F0001CC38280B70701401387074083A70740C5
:100A0000584B698F09C77D8D3335A0008280014521
:100A10008280B707014023AAA74082809C4513F734
:100A2000070113F8F70001C7D8413368E8008E21A9
:100A300013F7F50F39C318418146854E3D4F930F8B
:100A4000800293028004214E3396DE00B3F8C50085
:100A5000631116039398260033131F011343F3FF0A
:100A60003377E300B318180133E7E800639FF70515
:100A700050C98506E39AC6FD18C11307F00F6375C8
:100A8000B70454412146854E3D4F930F8002930297
:100A90008004414EB398CE0033F715016392E8020B
:100AA0001317260001173313EF001343F3FFB37638
:100AB000D3003317E800D98E639DF701232A15016F
:100AC0000506E319C6FD54C18280E39457FA10C9A4
:100AD0004DB7E39757FE23281501DDB708456D8D07
:100AE0003335A000828048456D8D3335A00082806B
:100AF0000CC9828019C20CC982804CC98280370718
:100B000000C0B377E5006395E708370701405C4311
:100B10009356B501584F9D8A9DE6F99BB70600FF95
:100B2000FD16758F89C993160501C182D58FB70649
:100B3000FF01758D498FB7060007D58FB7060140B5
:100B4000DCC2D8CE828005466396C600F59BB70608
:100B500080FFF9B709466396C600ED9BB706E8FF2C
:100B6000C1B70D466396C600DD9BB706FCFF4DBFBF
:100B700011466397C60093F7F7F3B706C0FF4DB76A
:100B80001546E391C6FA93F7F7CFB706E0FF49BFE2
:100B9000370700406391E702B7070140D84F42058D
:100BA000B367A70089E51345F5FFB377E50037077D
:100BB00001405CCF8280A9E337080140B7073000CD
:100BC0000326480013170501B376F50041836396A9
:100BD000F602B70600F9FD16B377D60003264800E3
:100BE000F18E2322D80091C5558112053315A70037
:100BF000C98F370701405CC382809317B50063D06B
:100C000007029357050193F6F7008D47B397D70076
:100C100093C7F7FFF18FB7060007D58FE9B7935752
:100C200055019207B317F700E5B713F7C50F93F710
:100C30003500B7050140BA9594458A073D473317FB
:100C4000F7001347F7FF758F98C598453315F500E2
:100C5000598D88C58280EFF2AFD137F4FF1F03278B
:100C600044723706003E4111931797019346F7FFF0
:100C7000F18F060737063E00718FD98F37060001C6
:100C800013979600718FD98FBD824167F98ED58FEA
:100C900002C202C402C623A0F182035784728545B2
:100CA000239CE180032704721305D00323A2E18271
:100CB0000327447023AEE180412C8327447037071B
:100CC0003A101307077093F7F7F06380E71063613A
:100CD000F70237073210130707706380E7063707FC
:100CE0003710130707706387E70841016FF08FCA59
:100CF00037073B1013070770638BE70A37073D1070
:100D000013070770E393E7FE85452165CD3BB714D4
:100D10000140E177130480044C00138504807C8239
:100D200022C6ED3985679387C7334C00138504C00D
:100D30007C8222C6E531F9770DA085452165C13356
:100D4000B7140140930700E0130480044C0013859E
:100D500004C07C8222C6D93189674C003715014016
:100D60007C8222C665398D477C8222C64C00138561
:100D7000044025A8B7140140E17793870770130456
:100D800080044C00138504807C8222C6413993077D
:100D9000D0E34C00138504C07C8222C64131F97730
:100DA0007C8222C64C00371501408D393DBFB714F7
:100DB0000140E177130480044C00138504807C8299
:100DC00022C6A939930740208DB7B7140140E177B7
:100DD000130480044C00138504807C8222C63D39B4
:100DE0008967F51799B723A4A182828003A781821E
:100DF000854714216310F7021C31639CE7023C21F4
:100E0000960793E707F837E700E093F7F70F369771
:100E10002300F740054793D756003317D7005441B6
:100E200089CE938707048A07B7E600E0B69798C390
:100E30008280EDF33C219607F9B793870706E5B763
:100E4000B7160240DC423747FF7F7D17F98F5D8D73
:100E5000C8C28280371702405C439146B18B638CD5
:100E6000D706A146638ED706BDE71C43918BA5C765
:100E7000B7470F00938707241CC1371602405C4216
:100E800037070020130707019183BD8BBA9794237E
:100E90001C41B3D7D7005CC15442A1829D8ABA9647
:100EA0009422B3D6D70014C55442AD829D8A36979A
:100EB0001423B3D6D70054C55842634C07005C4294
:100EC000B98313F7370093874180BA979C23B3D730
:100ED000F6021CC98280B7177A009387072069BF82
:100EE0005C435843C166C983BD8B758F8907C5466E
:100EF0006393D700C94701EF3747024003270780B4
:100F0000418B09CF37177A001307072021A837171D
:100F1000024058439316E700E3D606FE37173D001C
:100F200013070790B387E70281BF99C537170240BF
:100F30005C4B5D8D48CB8280B7170240D84B134580
:100F4000F5FF798DC8CB828099C5371702401C4FB9
:100F50005D8D08CF8280B7170240984F1345F5FF8B
:100F6000798D88CF828099C5371702405C4F5D8D9F
:100F700048CF8280B7170240D84F1345F5FF798DCF
:100F8000C8CF828099C5371702405C475D8D48C73E
:100F90008280B7170240D8471345F5FF798DC8C73F
:100FA00082801A218D6793870704B6217D8F9E2149
:100FB000D58FD621D58FF621D58F9625D58FB625FD
:100FC000D58FD625D58FF625D58FD98F1EA19E29F1
:100FD0001EA982801E2189C593E707041EA1828075
:100FE000C207C18393F7F7FBC207C183C5BF4EA5F4
:100FF00082804A2582800A256D8D3335A00082804B
:101000001E2137370140130707C0C207C1836300A1
:10101000E50237070040630CE5001307074063084B
:10102000E50037170040130707806316E500FA2133
:1010300093F7F7F8D98F9A2593F7F7CFC207C183B3
:10104000D98F371700401EA1130707809C416310FA
:10105000E5025CD5DE211EB5B7370140938707C096
:101060006314F500BC251EB985475EA98280C207BE
:10107000C1835EB5C5B71E31D22103D86500C20752
:10108000C183F99BC207C1831EB11E3156211A2D9F
:10109000C207C183420741831377C7F8518FB22536
:1010A000F59BC20633660601D18F37360140130621
:1010B00006C0C1826310C502D225DD9B03D805019D
:1010C000D18F9225ED9B93F6F6CFD18FF225336623
:1010D0000601D18E56A1B71600401AAD9386068040
:1010E00098416315D50058D91EB1828042074183CB
:1010F000DDBF1A31FD77FD17F98F1EB103580502C8
:1011000056215E2D6577D2211307F7CF7D8FF977B2
:101110002206FD17518FB3F70701F22103D8A5006E
:10112000C2064207336606013206D18F37360140C8
:10113000C207130606C0C1824183C183631AC5007A
:1011400071767D16F18EF2251A06D18EC206C18205
:1011500056A1B71600405AAD938606809841631594
:10116000D50038C11EB1828042074183DDBF1E21F8
:1011700089C593E717001EA18280C207C183F99B2E
:10118000C207C183CDBF8357450491C52167D98F5D
:101190002312F5048280C607C583DDBF5E2501C624
:1011A000DD8D4EA5828093C5F5FFFD8DDDBF1E212F
:1011B00089C593E707081EA18280C207C18393F700
:1011C000F7F7C207C183C5BF1E2DC207C183DD9BD0
:1011D000DD8D0EAD82805A2DFD779387F77FF98FD5
:1011E000A205CD8FC207C1835EAD8280B7170040D4
:1011F000938707806314F5002CC18280C205C181EA
:10120000E5BF1E294A25ED8F4205418189C76D8DB5
:101210003335A00082800145828093C5F5FFC20569
:10122000C1810EA98280EFE2BFF41629F577FD1780
:10123000F58FF621DA257971D58F1EA95625FD7710
:101240009387379FF58FD6212A842EC6D58F962572
:10125000D58FB625D58F5EA55E29C207C18393F7CA
:10126000F7CFD98F5EA96808F536B7470140938755
:101270000780B245631AF404A25756246547B38722
:10128000E702C206C186984163D2060406075224CB
:101290004206B3D7E702130740064186B3D6E702FA
:1012A000B3F7E7029206635506028E07938727037A
:1012B000B3D7E70213F77700B367D700C207C1833C
:1012C0001EA445616FE01FED925745BF0A07C1B7E5
:1012D000920793872703B3D7E702BD8BD58FF9BF5A
:1012E00091C55E250967D98F5EA582805A25F97759
:1012F000FD17F98FD5BF13F7F50F85471583B39504
:10130000B7006319F7009307C500984301CED98D44
:101310008CC38280894693074501E318D7FE930763
:101320000501E5B793C5F5FFF98DDDB793F5F51F19
:101330004EA182804A211375F51F82800A216D8D8E
:101340003335A000828013F7F50F85461583B397D8
:10135000B6006311D7025A25F98F1A2101454207B9
:10136000418381CB0545A181B315B5006D8F333520
:10137000E000828089466314D7001A29F1BF5A29F8
:10138000E1BFEFE2FFDE7971130600028145080834
:10139000EFE01FE18545114502C202C402C66D3669
:1013A0008545130500204D360145593C3715014050
:1013B0009307E00F4C0013050580372401407C8221
:1013C00002C6EFF0AFE513050440EFF0EF8F130511
:1013D0000440EFF0EFABAA852396A18237550000B9
:1013E00013050551EF201074B7070E003ECE0C0810
:1013F0008547130504402302F10202C802CA02CC49
:1014000002D0EFF0EF8E854513050440EFF0AF9367
:10141000854513050440EFF08FA581451305044071
:10142000EFF04FA213050440EFF00F949304044033
:101430002685EFF00F946DFD13050440372401401D
:10144000EFF0AF93930404402685EFF0AF936DFD6A
:1014500037050080F532130504408545EFF00FA0F5
:101460009305000213050440EFF08FA145616FE082
:101470007FD2EFE2FFCF39711306C0022A89AE8412
:1014800048088145EFE0DFD1854505453704024036
:1014900002C602C8593C13058400EFF00FBDB72700
:1014A00001409387C7443ECA930700083ED4930780
:1014B00000103ED6930700403ED8930700023EDA64
:1014C0004C088D67130584003EDC4ACC26D002CE42
:1014D00002D202DEEFF08FC3054689451305840072
:1014E000EFF08FC7ED477C8685475C8768008547AE
:1014F0003EC8EFF0BF8F854513058400EFF08FC421
:1015000021616FE03FC9EFE2BFC6AA842E84056562
:1015100001118545130505807D1402C602C802CA63
:1015200002CC02CE02C002C202C4393C608237340F
:1015300001408A85130504C0FD1426C02314010050
:1015400023130100753CA9473EC6C1679387070670
:101550003EC86C008947130504C0FC83293E13056F
:1015600004C085450D31130504C08145B13913050B
:1015700004C085452D398545130504C0CD3E056160
:101580006FE05FC1EFE2DFBE7971130600028145B3
:101590000808EFE0FFC08545114502C202C402C63B
:1015A000EFF09F9A854513050020EFF0FF99014564
:1015B000EFF01F89371501409307E0074C00130532
:1015C0000580372401407C8202C6EFF02FC5130549
:1015D0000440EFE07FEF13050440EFF06F8B23969C
:1015E000A18285473ECA0C0899471305044023028F
:1015F000F10202C802CC02CE02D0EFE07FEF8545B7
:1016000013050440EFE03FF5854513050440EFE086
:101610009FF3854513050440EFF06F858145130561
:101620000440EFF02F8213050440EFE0FFF3930432
:1016300004402685EFE0FFF36DFD130504403724D9
:101640000140EFE09FF3930404402685EFE09FF311
:101650006DFD13050440954605468545EFE01FF3F3
:1016600013050440954609468945EFE03FF213050E
:10167000044095460D468D45EFE05FF113050440AB
:10168000954611469145EFE07FF0130504409546DD
:1016900015469545EFE09FEF954619461305044022
:1016A0009945EFE0BFEEB165938505B87945A13D59
:1016B000994513854186753B45616FE0BFAD41118A
:1016C000094522C6EFF04FAB05C50945EFF06FABFA
:1016D000138441862E203755000013058552EF20D4
:1016E00070444E20375500001305C552EF2090433B
:1016F0003244410173002030EFE29FA7011185457C
:101700002145EFF07F8485451165EFF0DF853714C3
:10171000014085678D447C808A85C147130504C0DC
:101720003EC426C2EFF08FAF130504C08565EFF00D
:101730002FBC896761498A85130504C07C804AC42F
:1017400026C2EFF0AFAD91677C808A859147130583
:1017500004C03EC4EFF08FACE1778A85130504C066
:101760007C804AC426C2EFF06FABB70704013EC6C7
:10177000B70702003EC8B70700028507374400409C
:101780003ECAA1473ECC6C009D4713050480FC86F1
:10179000EFF03F81854513050480EFF0BF830561BD
:1017A0006FE05F9FEFE23F9BB74400402A8913043C
:1017B000900C9389048089454E85EFF0DF8305C93D
:1017C000CA8513850480B7440040EFF05F8213049C
:1017D000900C1389048085454A85EFF0DF8119CD8F
:1017E00013850480EFF0FF801375F50F31A07D1491
:1017F0001374F40F69F001456FE03F997D14137481
:10180000F40F71F8CDBFEFE2BF962A89371501407A
:101810002E84130505C08565B2840146EFF08FADB7
:101820000D454937135504011375F50FA53F1355A1
:1018300084001375F50FBD371375F40FA5370144F8
:1018400093170401C18363EC9700371501400546E7
:101850008565130505C0EFF0EFA96FE0BF93130591
:10186000F00F8937B307890088A30504D1BFEFE2E1
:101870003F90411185451145EFF00FED854521451C
:10188000EFF08FEC930700107C8237150140C147C1
:101890003EC64C008D47130505803EC4EFF00F98FF
:1018A00041016FE03F8FEFE2BF8C4111854541451B
:1018B000EFF08FE98567938707807C8237150140B9
:1018C000C1473EC64C008D47130505803EC4EFF06E
:1018D000EF9441016FE01F8CEFE29F894111854534
:1018E0002145EFF06FE693070010371401407C822A
:1018F000C1473EC64C008D47130504C03EC4EFF0FF
:10190000EF91014693050010130504C0EFF08F9E80
:1019100041016FE03F88EFE2BF857971854525453C
:10192000EFF08FE2914737150140FC824C08930796
:101930008004130505C03ECEEFF04F8E8945054566
:10194000EFF0AFAE914705443ED00810B1473ED40A
:1019500022D602D2EFF06F83930780117C86680055
:1019600089475C8722C8EFF06FC845616FE09F82AE
:101970004111114522C6EFF0EF8785476315F50247
:101980002A841145EFF0EF8803C7E18409EFB725FA
:10199000000081461306803E9385C5331385018C74
:1019A00023878184E1293244410173002030EFE232
:1019B0002FFC797185451545EFF00FD985673715EF
:1019C0000140FC824C0893078002130505803ECE3F
:1019D000EFF0CF84B1450145EFF02FA585670544B1
:1019E0003ED00810A1473ED422D602D2EFE0FFF944
:1019F000930780137C8668008D475C8722C8EFF0D0
:101A0000EFBE45616FE00FF90565EFE0BFFE85476A
:101A10006314F5020565EFE0DFFF83C70184B72596
:101A20000000850781461306803E9385253A13857D
:101A3000018B2380F184992173002030EFE24FF372
:101A4000411185452145EFF02FD085451145EFF037
:101A50008FD193070020371401407C82E1473EC6B6
:101A60004C008D47130504C03EC4EFE03FFB9307D5
:101A700000084C00130504C07C82EFE03FFA4101EE
:101A80006FE04FF1EFE2CFEE01114D3F3714004010
:101A90009307F01D8A85130504803EC002C22314FB
:101AA000010023050100EFF0AFD513050480854543
:101AB000EFF0EFEFC167938707066C001305048012
:101AC0003EC8231B010002C6EFF0AFE213050480FD
:101AD000A145EFF04FF0130504808545EFF02FE9A5
:101AE000854513050480EFF00FEA05616FE08FEA8A
:101AF000411122C42A8408414AC24EC006C6EF20C2
:101B0000004FB757000003A6075483A647542A89FD
:101B1000AE89EF00B04B635F0502B757000083A7A3
:101B200047531CC0B757000083A5C7530840EF10A8
:101B30001058EF2080399315050137150040C181F9
:101B400013050580EFF08FEAB24022441249824922
:101B500041018280B757000003A6875483A6C7546B
:101B60004A85CE85EF00B03BE35EA0FAB757000090
:101B700083A787537DB7EFE2AFDF79713714014058
:101B8000C1472A89FC828D44C1474C08130504C013
:101B90003ECE26CCEFE09FE80146130504C0C145C8
:101BA000EFE05FF585452145EFF00FBA8545370534
:101BB0000800EFF04FBB8547FC824C08E147130556
:101BC00004C026CC3ECEEFE07FE5894491474C0827
:101BD000130504C0E482375400403ECEEFE01FE41A
:101BE0000C10B7070C00130504C04AD03ED402D233
:101BF00023160102EFF02FE39307D0137C866800D1
:101C000085473EC84487EFF06F9E0546130504C024
:101C100093055052EFF02FEE8545130504C0EFF009
:101C20002FEC45616FE00FD7EFE28FD47971371455
:101C30000140930700022A89FC828D44C1474C0869
:101C4000130504C03ECE26CCEFE05FDD0146130550
:101C500004C093050002EFE0FFE985452145EFF060
:101C6000AFAE854537050400EFF0EFAF93070040B6
:101C7000FC824C08E147130504C026CC3ECEEFE0C1
:101C8000FFD9856793870780FC824C08914713052D
:101C900004C03ECE37540040EFE05FD80C10B707C9
:101CA0000C00130504804AD03ED402D22316010250
:101CB000EFF06FD7930770137C8685475C876800C9
:101CC00085473EC8EFF08F920546130504809305C3
:101CD0005052EFF04FE2854513050480EFF04FE0DE
:101CE00045616FE02FCB411122C637540040930568
:101CF000505213050480EFF00FE50DC51305048065
:101D0000EFF04FE39375F50F2388B18203A541856A
:101D10001C4D104954498507B3E7C7026384D700B7
:101D2000310505243244410173002030411122C69F
:101D30003754004093055052130504C0EFF0AFE054
:101D40000DC5130504C0EFF0EFDE9375F50F238A80
:101D5000B18203A581851C4D104954498507B3E71D
:101D6000C7026384D7003105E92A32444101730078
:101D70002030411122C63704004085451305044038
:101D8000EFF02FC819C5854513050440EFF0EFC8E3
:101D9000B9293244410173002030EFE26FBD0111D7
:101DA0002E84AA8485450545EFF0EF9B4C08370546
:101DB000004026CAE084231E0100231D0100EFF02D
:101DC0002FA40546854537050040EFF02FBD93074A
:101DD000C0027C868D475C87680085473EC8EFF06F
:101DE000EF80854537050040EFF06FB805616FE083
:101DF0006FBAEFE2EFB7B707002083A50710896736
:101E000093870771B3D5F502A9473305F502FD1590
:101E1000C205C1817D154205418141376FE08FB711
:101E2000854537050040EFF0CFBD19C5854537051D
:101E30000040EFF08FBED12873002030B7F700E0EC
:101E400023A20700D92073002030411122C6373465
:101E500001408545130504C0EFF0AFBA01CD13056D
:101E600004C08545EFF06FBB3755000013050555DD
:101E7000EF20805C32444101730020301DC9B296CE
:101E8000C206C18252A136A10CC509EE85471CA12C
:101E900083A6818393878183368701EB54C588C3EA
:101EA0000145828023000500E5B76306A700584777
:101EB000EDB77D558280054582800DC583A781835E
:101EC0001387818399E305458280D4476396A600F2
:101ED0005845D8C7014582806394A70014C3DDBF6D
:101EE000B687CDB77D558280EFE28FA803A48183AA
:101EF00075DC1C2093F7F70F99C75E2099C3230068
:101F000004001C4482974044E5B783A781830546BB
:101F100091E38280D62381CEBA237D174207418385
:101F2000BAA3BA234207418319E390A3B6A3DC47BF
:101F3000C5B7232605000CC150C123240500054563
:101F400082805C45544118458507B3E7D702638E0C
:101F5000E70058451C41BA978CA35C45584185075A
:101F6000B3E7E7025CC50545828079558280B707F3
:101F7000002083A707100967130707F4B3D7E70208
:101F8000C207C183239FF182239EF1828280EFE208
:101F90002F9E2A841165011185451105EFE0DFFAB6
:101FA000930700207C82371501408D473EC44C00CA
:101FB000E147130505803EC6EFE05FA622C837441F
:101FC0000140B70708000C08130504803ECC02CA84
:101FD000231E0100EFF02FA5854513050480EFF0C7
:101FE0002FB005616FE00F9BEFE2EF96B744014021
:101FF000AE893289014493840480634524014A8573
:102000006FE0AF98930500042685EFF02FB37DD9DC
:10201000B38789008385070026850504C205C18131
:10202000EFF0CFB0D9BF138781801C43938681AE78
:102030003E95636BD500B75600209386068063E516
:10204000A60008C33E858280FD57EDBFEFE24F92A8
:10205000138701872A2383D701873355F502EF10B1
:10206000306CB757000083A50756EF1050046FE09F
:102070006F92EFE2EF8F138701874A2383D701879F
:102080003355F502EF10D069B757000083A5C75745
:10209000EF10F0016FE00F90EFE28F8D1387018753
:1020A0006A2383D701873355F502EF107067B7575E
:1020B000000083A50756EF10807F6FE0AF8DEFE241
:1020C0002F8B138701870A2783D701873355F502A2
:1020D000EF101065B757000083A58757EF10207DDC
:1020E0006FE04F8BEFE2CF88138701872A2783D7D2
:1020F00001873355F502EF10B062B757000083A592
:10210000C757EF10C07A6FE0EF88138701875A270F
:1021100083D7018701459306100F3357F702956760
:10212000938707589223636AC702EFE26F84EF1028
:10213000A034B757000003A6875683A6C756EF0002
:102140004074B757000003A6075783A64757EF0010
:10215000D03EEF1090746FE0EF8305058907E3131D
:10216000D5FC130500008280EFE28F803971680092
:10217000130620038145EFF00FE918869307300519
:10218000370500206317F70298869307C00463128F
:10219000F7020347D103D947631DF7001306200355
:1021A0006C0013050502EF20C00C054521616FD0BE
:1021B0007FFEB707002003C7470513050502938775
:1021C000470518A1983318B1B82338A1B83338B1EE
:1021D000D82358A1D83358B1F82378A1F83378B16F
:1021E0009827DC3718A5A308F5020145C1B7EFD23F
:1021F0003FF8A93D138401889357850048B87CA80F
:102200009357050161817CB808AC793593578500F7
:1022100008BC3CAC9357050161813CBC48AC913D86
:102220009357850048B47CA49357050161817CB421
:1022300008A84D3D9357850048BC7CAC93570501D9
:1022400061817CBC2300A402C93593578500A30299
:10225000A4022303F402935705016181A303F4024E
:102260002304A402A93D935785002301F402935748
:102270000501A301F402A300A40223980186618151
:10228000938701872302A40223910700239207006A
:102290002393070023940700239507002396070044
:1022A0006FD05FEFEFD2DFEC938701859843D5665F
:1022B000938606186307D702050798C337140140B1
:1022C000856493850480130504800546EFE09F82B2
:1022D00001469385048013050480EFE0BF816FD031
:1022E0007FEB23A00700B707EFBE37E700E0938737
:1022F00007083CC7E1B7EFD2BFE79387118490236B
:10230000371401409305001013361600130504809E
:1023100090A3EFE02FFE138791841C23850793F78A
:10232000F70F1CA329476399E700054693050010A2
:10233000130504C0EFE00FFC6FD0DFE51387A18425
:102340001C233706002013060602850793F7F70FB4
:102350001CA38346C6028345B602A206CD8E6391B6
:10236000D704EFD2FFE01384018C1385018C230086
:10237000070023870184EFF05FB4230004003714C3
:1023800001409145130504C0EFE04FF501E9014616
:1023900093050010130504C0EFE0CFF56FD09FDF69
:1023A0008280EFD2FFDC03C7E18485471384B184C8
:1023B000938401846310F7021389018B1385018BC9
:1023C000230004002396018423800400EFF0FFAE75
:1023D00023000900982085476315F7001C20850716
:1023E0001CA0370900209306090283C7E60203C632
:1023F000D6021420A207D18F130909026390F602B6
:10240000230004001384018B1385018B23800400B7
:10241000EFF0BFAA230004006FD0DFD7854763FD2C
:10242000E70037150140014693050010130505C06C
:10243000EFE04FEC23000400371501409305001036
:10244000130505C0EFE02FEA9387C18401E59A23C5
:1024500005079AA3034709030346F90296232207B7
:10246000518FE39BE6FA37150140054693050010AE
:10247000130505C023900700EFE0CFE761B7EFD267
:102480009FCDB70400209384040283C7240203C5B0
:102490001402A2075D8DEF10B028B757000083A586
:1024A000877613840188EF104004BC20938941840F
:1024B000370700203CA0BC30130747052380018864
:1024C0003CB0DC20A380018823A0A9005CA0DC3004
:1024D000138901885CB0FC207CA0FC307CB09C247B
:1024E0001CA43C271437A207D58F1CB4A1833CA49D
:1024F0005C273437A207D58F3CB4A1835CA4EFF0EE
:102500005FB79357850048B47CA493570501618158
:102510007CB408A8EFF09FB39357850048B87CA817
:102520009357050161817CB808ACEFF0FFB6935773
:1025300085015CAC7C24443413578500A207C58F09
:10254000643438AC13570501C204C58F042838BC65
:102550005838E204DD8C7C28AA8508BCA2075D8F70
:102560007C38C207D98F182C62073365F700EF104B
:10257000405D83A50900EF108033AA852685EF1002
:10258000405C9357850008B83CA8935705016181CA
:102590003CB848A8EFF0BFB293578500A300A4024F
:1025A0002301F402935705016181A301F402230280
:1025B000A402EFF09FB5935785002303F4029357CD
:1025C0000501A303F4023C280438A302A402A207D5
:1025D000C58F243861812304A402C204C58F442816
:1025E000E204DD8CB757000083A547772685EF10FE
:1025F0004023634B0500B757000083A50777268566
:10260000EF10C0196355A00005472384E184B71477
:10261000014093050010138504C0EFE0CFCC814743
:1026200001C99145138504C0EFE04FCBB337A0003B
:10263000A304F90223050902A305090223060902DE
:102640006FD0BFB4EFD2DFB2EFF01FB2EFF03FE3D5
:10265000B725000081461306803E9385652F1385BC
:10266000018DEFF0BF81B7250000F9461306803ECB
:102670009385452A1385018EEFF05F80EFF0DF86AA
:102680006FD05FB1EFD2DFAE0545EFF08FF63D289A
:10269000EFF04FBFEFE0FFCEEFF06F9DEFF0AFA098
:1026A000EFF08F85EFF04FA3EFF0EFA6EFF02FB034
:1026B000EFE05FEDB757000083A7877723A6F1808F
:1026C0001385C180EFF0CFC26FD0DFACEFD25FAA2D
:1026D00037040020130444061306800C9385018FF1
:1026E0001305C400EFF0FF84716513050520EFF0BA
:1026F000AFD3854404A01306C0129385819B1305B4
:10270000840223AA8184EFF0DF8248507104EFF045
:102710008FC604A0014523AC81846FD0BFA713D717
:102720004501B7071000FD1713D846011377F77F4F
:102730009308F07F33F3B7002A8EF58FFD81B28EB8
:102740001378F87FFD8263081703630018030DEB0D
:10275000B368A300631408005D8E29CA638508046A
:102760006388D502054595ED8280B3E8C700E38014
:1027700008FE795582803365A30065FD630CE8028D
:10278000631408005D8E79DEE39ED5FCE34CE8FC23
:1027900063480701E3E867FC6303F302637FF30028
:1027A00081E57D558280F5DE054582800145E39B0C
:1027B00008FA82805D8E69DA6DBF01458280E3E3AD
:1027C000CEFB0145E372DEFBE5F1E1BF13D7450126
:1027D000B7071000FD1713D846011377F77F93084A
:1027E000F07F33FEB700AA8EF58FFD81328F13780C
:1027F000F87FFD82630E1703630D180129E3B368A8
:10280000AE00631F08005D8E01EE0143638C080477
:1028100021A8B3E8C7000943639608046DD305A057
:10282000638408046385D50205438DCD7D531DA8BF
:10283000B368AE00094363970802630AE8026314B1
:1028400008005D8E75D2E391D5FEE34FE8FC634945
:102850000701E3EBC7FD630FFE0001436374FE0055
:10286000F1D505431A858280EDFE7D53E5BF5D8E6F
:1028700079DACDBFE36ADFFB0143E3F5EEFFF5F163
:1028800075B739714AD813D945014ED652D456D2AC
:102890009399C50006DE22DC26DA5AD05ECE137983
:1028A000F97F2A8A93D9C90093DAF501630D090EDD
:1028B0009307F07F6306F9181354D5018E09B369A5
:1028C00034013704800033E4890093143500130980
:1028D00019C08149814B13D74601139AC60013775B
:1028E000F77FB285135ACA0013DBF601630B07109A
:1028F0009307F07F6303F7049357D6010E0A33EA78
:102900004701130717C0B7078000B367FA00931594
:1029100036003A99814833C76A01BD463A851308A3
:10292000190063E8361717360000130666E58A09B2
:10293000B29983A60900B2968286B367CA001309CA
:10294000F97F6399071293E9290081458948E1B726
:1029500001479307F07F3704080081443204D2070F
:1029600031807E075D8C598CA285F2506254268599
:102970004259D254B259225A925A025BF24B216107
:1029800082805A853E84AE84C68B8947638DFB0E58
:102990008D47E38FFBFA85472A87639EFB38814783
:1029A0000144814465BF33E4A90061C036C632C426
:1029B000638C092A4E85EF10F0042246B246AA879E
:1029C000130755FF7544938487FF198CB3999900B9
:1029D00033548A0033643401B3149A0013D7460188
:1029E0001309D0C0139AC6001377F77F3309F94053
:1029F0008149814BB285135ACA0013DBF601E319F2
:102A000007EEB367CA00B1C7630F0A22528532C40A
:102A1000EF10407F22462A87930655FFF54793051E
:102A200087FF958F331ABA00B357F600B3E7470113
:102A3000B315B6003309E9401309D9C08148E1BD97
:102A400033E4A90001ECA14981441309F07F894BCB
:102A500059B593E919008145854875BD4E84AA840E
:102A6000B1491309F07F8D4BBDB5914981440149AE
:102A7000854B95B593E93900D2878D4869BD894763
:102A80005685E397FBF02A879307F07F0144814442
:102A9000F1B5C16E1386FEFF93D6040113DE050166
:102AA000F18CF18D338695023383B602935806017B
:102AB00033059E021A95AA98B382C60363F3680091
:102AC000F692C16F1383FFFF33F5670093D30701BD
:102AD000B3F76800C207337366003E93330695026E
:102AE00093D80801B387A602135F0601B38493024B
:102AF000BE94FA94B38E760263F3F400FE9E416AAC
:102B00009307FAFF935F0401B376F400B3F9F4007E
:102B10007D8EC1803384D502C209338FD401B2992E
:102B2000CE98B307DE02935E0401B385BF02AE9771
:102B3000BE9E330EFE0363F3BE00529EC1679385B3
:102B4000F7FF33F6BE006D8C4206229693DE0E012F
:102B5000B305D502769E3385AF0213D40501B38643
:102B6000D302AA96A296B38FF30363F3A600BE9F87
:102B700041657D15B3F7A600C2076D8DAA97B38591
:102B80005800B3B93501FA97B2953384370133B69B
:102B9000C500B30EC4013385CE0033343401B3B75E
:102BA000E701C18F33BECE0113D406013336C50011
:102BB0003E943366CE009394950032947E94B3E4B1
:102BC0006400260493567501B3349000DD81931799
:102BD0009500CD8C558CDD8C9317740063DB07005A
:102BE00093D7140085889316F401DD8CD58C05806D
:102BF00042899307F93F6359F00893F6740081CE38
:102C000093F6F40011466388C60093864400B3B47B
:102C100096002694B6849316740063D80600B7070E
:102C200000FFFD177D8C930709409306E07F63CF7B
:102C3000F60E93D634009314D4012604D58C31803B
:102C400093F7F77F21BB328532C4EF10A05B930668
:102C50005501F147130705022246E3D1D7DC611580
:102C6000B317A6008145F9B3EF10C05913075501FA
:102C7000F145930705022246B246E3D5E5D4611536
:102C80003314AA00814499BB85469D8EB1E7130990
:102C9000E941B3972401B3D4D40033192401B337E5
:102CA000F000B3649900DD8C93F77400B356D40040
:102CB00081CF93F7F40011466388C70093874400DF
:102CC000B3B49700A696BE849397860063D8070492
:102CD00085470144814459B113068003E341D6CCB2
:102CE0007D46E356D6FA0556B307F6409305000233
:102CF0003356F4006387B6001309E943B317240180
:102D0000DD8CB3349000D18C93F67400014499CAE1
:102D100093F7F40011468146E392C7FA13949600A4
:102D20003180F6068D80D58C81470DB99307F07FF1
:102D30000144814425B142896DBD370710007D17DC
:102D400001113373B70093D84601758F935ED60196
:102D500022CC26CA0E0393D445019357D5010E0702
:102D600006CE4AC84EC693F8F87F130EF07F33E7BD
:102D7000EE0093F4F47F13D4F50133E36700131FDF
:102D80003500FD82931E36006380C81993C6160075
:102D9000B38514416305D4126351B018638B081ACC
:102DA000B70780005D8F6381C4599307800363C4B4
:102DB000B734FD4763C5B748930700028D8FB3D979
:102DC000BE003318F700B39EFE0033683801335756
:102DD000B700B339D001336838013303E340B30996
:102DE0000F41B3373F013306F3409317860063D397
:102DF0000724370980007D1933792601630F092CD8
:102E00004A85EF102040130785FF93070002998F32
:102E1000B3D7F9003316E900D18FB399E9006344C1
:102E2000972A058F13061700FD4663C5C63A130798
:102E30000002118FB3D6C9003398E9003397E70039
:102E4000558F33380001B369070133D6C700814479
:102E500093F7790081CF93F6F90091476388F600E4
:102E60009386490033B836014296B6899317860097
:102E700063D6071C138714009307F07F0588630649
:102E8000F720B70780FFFD17F18F1398D70193D96B
:102E90003900A60733683801B1831377F77F93961B
:102EA000C7005207B1827E04D98EC18EF2406244BF
:102EB000D2444249B2494285B68505618280635653
:102EC000B00A638A0812B70780005D8F6387C42D3C
:102ED0009307800363C7B718FD4763D2B73C1388D5
:102EE00005FE93070002B3590701638AF5009307B3
:102EF0000004B385B7403317B700B3EEEE003338A4
:102F0000D0013368380195A2B367D7019385148047
:102F100099E393C61600630AD404D1E193871400A1
:102F200093F7E77F6399071EB367E3013368D7011F
:102F3000639204166382073C631608421318350037
:102F40009316D3011358380033E806019357330022
:102F500019A2B367D7016385071A9387F5FF638BBF
:102F6000073A638CC523BE8589B56399051C938692
:102F7000140093F7E67FC1EFB367E3016390043673
:102F8000638D0744B367D701639407460E05131892
:102F9000D3010D813368A800935733006DA8B38522
:102FA000984063970420B367E301638D07309387EC
:102FB000F5FF638907401305F07F6383A520BE8575
:102FC0009307800363C2B72AFD4763C8B73C9307E2
:102FD00000028D8F3318F3003356BF00B317FF0084
:102FE0003368C800B339F0003353B3003368380195
:102FF00033076740B5ACB367D70163830710938786
:10300000F5FF638F071E6380C52FBE85D1B593077B
:10301000F07F638BF606FA9E33B6EE01B307E3004A
:10302000B2971398F70193DE1E00B369D80113D647
:103030001700B68493F77900E39F07E09317D60152
:1030400013D839003368F800A68593573600130764
:10305000F07F6380E506B207B18313F7F57F05883B
:103060003DBD3367D7013338E000B309E801B3B79A
:10307000E9013386670093178600E3DD07FA8504CC
:103080009307F07F639CF41805881307F07F81474E
:10309000014831B5639107106301083C13183600ED
:1030A0009317D701135838003368F80036849357C4
:1030B0003700B367F800E9DB01441307F07FB70777
:1030C00008000148E9BB370680FF7D167D8E93F727
:1030D0007900998CE39107D895B74E85EF1080124F
:1030E00013078501FD47E3D2E7D2130685FFB397A7
:1030F000C90081492DB33368D70133380001C5B108
:10310000131835009317D301135838003368F800AB
:10311000935733002DBFB309DF413309E340333602
:103120003F013309C9409317890063CA072033E878
:103130002901E31508CC8147014431BFB38598408C
:1031400063810414B70680009307F07F3363D300D4
:103150006381F8209307800363CCB722FD4763C9DE
:10316000B72C930700028D8F3318F300B356BF00BE
:10317000B317FF003368D800B339F0003353B300FE
:10318000336838011A97B309D801B3B7D901338628
:10319000E700C684CDB5E31108F213183500931784
:1031A000D301135838003368F8009357330011B730
:1031B000370580009307F07F3363A300E392F8E0C4
:1031C0000E061318D7010D823368C80093573700D5
:1031D0003684C5B505179306000233D7E700630AA6
:1031E000D600930600043386C6403396C700B3E981
:1031F000C90033383001B369E800014681441DBD80
:10320000B309DF01B307E30033BFE9013386E70108
:10321000931786008544E3DF07E08944B70780FF02
:10322000FD17F18F13D7190013F819003368070140
:103230009399F701B3E9090113D6170011B913885F
:1032400005FE93070002B3590701638AF50093074F
:103250000004B385B7403317B700B3EEEE00333840
:10326000D00133683801A5BE3363E3013338600011
:10327000B3890E41B3B73E013306F740C6843684A6
:10328000ADB6B367E301638707189387F5FF638CD7
:10329000071C9306F07F638ED50ABE8565BD930734
:1032A00000028D8FB3D9BE003318F700B39EFE0025
:1032B000336838013357B700B339D0013368380168
:1032C0003A9365B3131836009317D7011358380093
:1032D00033E8070136849357370095BBBDCB33677E
:1032E000D701E31B07DC0E051318D3010D813368EA
:1032F000A8009357330075BBE30F08E2131836009C
:103300009317D701135838003368F8003684935761
:10331000370091B3B309DF41B307E340333F3F01C7
:103320003386E7418544D1B4131835009316D30191
:103330001358380033E80601935733009DBBB38917
:10334000EE413306674033B93E01330926413684E6
:1033500075B40E061318D7010D823368C800935751
:10336000370081BBB309DF41B307E34033363F0188
:103370003386C7409317860063D7070AB389EE41A7
:10338000B3076740B3BE3E013386D7413684C9B424
:103390003363E30133386000FDB3138805FE930700
:1033A0000002B3590301638AF50093070004B38553
:1033B000B7403313B300336F6F003338E001336825
:1033C00038017DB5B389EE41B3076740B3BE3E0116
:1033D0003386D7413684854409BC131836009317C9
:1033E000D701135838003368F80093573700A5B158
:1033F000B309DF01B307E30033BFE9013386E70117
:1034000093178600E3D807C2B70780FFFD177D8EAC
:1034100085440DB10E061318D7010D823368C8001C
:10342000935737002DB133E8C900E30608D019B12E
:10343000138805FE93070002B3590301638AF50060
:1034400093070004B385B7403313B300336F6F00A5
:103450003338E001336838013DB301441307F07F8E
:10346000B70708002DBCB309DF01B307E300B3BE03
:10347000D9013386D70169BB411106C622C426C2D1
:103480000DCD9357F541B3C4A7009D8C2A842685A2
:10349000EF0050579306E041898EA9477D8093F64F
:1034A000F67F63CDA7022D47098FB3D7E4005505FA
:1034B000B207B394A400B18329A001448146814797
:1034C0008144B207D206B1837E04D58FC18FB2404A
:1034D00022442685BE859244410182805515B397CA
:1034E000A400B207B1838144E9BF397193577501D4
:1034F0004AD856D25ECE931A95001359F50106DECE
:1035000022DC26DA4ED652D45AD093F7F70F93DA4C
:103510009A00CA8B638207121307F00F6384E712C5
:103520008E0A37070004B3EAEA00138A17F8014449
:10353000014B93D775019394950093F7F70FA580EE
:1035400093D9F501FDC71307F00F6387E7028E04D7
:10355000938717F837070004D98C330AFA4081465D
:10356000558C172700001307A7250A043A941C401E
:1035700033493901BA978287130A1AF0F9E8894664
:10358000558C172700001307A7270A043A941C40FC
:1035900033493901BA97828701491307F00FB707FA
:1035A000400013959700F2506254931777012581DC
:1035B0007E095D8D33652501D2544259B259225A94
:1035C000925A025BF24B216182801307F00F814710
:1035D000C9BFA68ACE8B368B8947630BFB1A8D47F2
:1035E000E30CFBFA8547630AFB0A1307FA0713F992
:1035F0001B006357E01293F77A0099C793F7FA001C
:1036000091466383D700910A93974A0063D90700D4
:10361000B70700F8FD17B3FAFA0013070A08930773
:10362000E00FE3C4E7FA93976A00A5831377F70FD7
:103630008DBFB9E48546A9B763940A021144014AD3
:10364000054BC5BD63990A002144130AF00F094BCD
:10365000CDB58D4631B73144130AF00F0D4BD1BDB6
:1036600056852EC6EF00103A9307B5FFB39AFA00BD
:103670009307A0F8338AA7400144014BB24555BDDA
:103680002685EF0030381307B5FFB307AA00B394BF
:10369000E400138A67078146E1B513F91B0001476F
:1036A000814701B74166139554007D169357050174
:1036B000698E63FA9A0AB3D5FA027D1AD686014753
:1036C0003388C502B3F6F602C206558F637B070145
:1036D0002A979386F5FF6368A70A6376070BF915A7
:1036E0002A9733070741B356F7023377F702B38AB5
:1036F000C6029317070163FB5701AA971387F6FFCA
:1037000063E1A70863FF5707F916AA97C205B38AB2
:103710005741D58DB33A5001B3EA5501CA8BF1B583
:103720008546998E11C76D4601478147E34BD6E622
:10373000130AEA09339A4A01B3D7DA00B33A4001CF
:10374000B3E7570113F7770019C713F7F70091464E
:103750006303D700910713975700634807029A073E
:10376000A58301473DBD93D61A00B3D5F602139742
:10377000FA0141833388C502B1B7CE8B368B814ABB
:10378000A1BDBA8661B7B685A9BF0547814711BDFE
:1037900013F91B001307F00F814721B593567501EC
:1037A000B7078000FD1713D6750193F6F60F1308BF
:1037B000F00FB3F8A7001357F501ED8F1376F60F4E
:1037C000FD8163810603630C06018DE211E2B1C342
:1037D000638E08026305B70405451DE78280F5D7AF
:1037E00079558280E39E08FE6309D60211E2EDD787
:1037F000E314B7FEE342D6FE63C7C600E3EE17FD4F
:103800000145E3FDF8FC01E77D558280F5DD0545C6
:1038100082800145E39208FC8280F9DBD1B78146C2
:10382000E1BF93567501B7078000FD1713D67501E8
:1038300093F6F60F1308F00FB3F8A7001357F5012E
:10384000ED8F1376F60FFD8163870603630906018A
:1038500085EA11EA89EB0145639B080082800945EE
:10386000F5FFE5DA31A8638C08026300B70405456B
:1038700075D77D5582800945639808026304D60296
:1038800011E2F5D7E315B7FEE343D6FE63C7C600E2
:10389000E3EF17FD0145E3F3F8FC19E3D9BFF1D9D4
:1038A00005458280E5D3828082808146C5B77971E3
:1038B00022D4135475014ECE52CC9319950006D6DE
:1038C00026D24AD056CA5AC81374F40F93D9990015
:1038D000135AF50169C49307F00F6308F40E939728
:1038E000390037070004B3E9E700130414F88144F2
:1038F000014B13D77501939A95001377F70F93DA5D
:103900009A0013D9F50145CF9307F00F630CF70226
:103910008E0A130717F8B7070004B3EAFA003A94BF
:10392000014633452A01BD47AA869305140063E288
:103930009710172700001307A7F08A04BA949C4039
:10394000BA9782871304F40F63980A0C93E4240057
:103950000946C1BF01451307F00FB7074000B25039
:103960002254A6075E07A5837E05D98F925402597B
:10397000F249624AD24A424B5D8D45618280CA86D5
:10398000D689328B89476301FB0A8D47E304FBFC30
:10399000854736856312FB1A01478147C9B7639E85
:1039A000090413D77501939A95001377F70F914483
:1039B0000144054B93DA9A0013D9F50131F7639D61
:1039C0000A0093E414000546A9BF63930902A144C9
:1039D0001304F00F094B31BF5685EF00B002930777
:1039E000B5FF098CB39AFA001304A4F8014615BF79
:1039F000B1441304F00F0D4BEDBD4E852EC6EF0004
:103A000070009307B5FF1304A0F8B399F900098C6F
:103A10008144014BB245F1BD93E434000D4611B72A
:103A20008947D286E313FBF636851307F00F8147EB
:103A30003DB741639306F3FF13D6090193D80A01FA
:103A4000B3F7D900B3FADA0033885703B389F80221
:103A500013570801B30A5603D6994E973306160337
:103A6000637357011A96C167FD17B376F700337871
:103A7000F800C206C2969399660093570701B339BE
:103A80003001E982B2979A07B3E6D900B3E9D700CB
:103A90009397490063D9070013D7190093F71900CA
:103AA000B369F7002E841307F4076350E00493F71B
:103AB000790099C793F7F90091466383D70091097C
:103AC0009397490063D90700B70700F8FD17B3F9CA
:103AD000F900130704089307E00F63CBE7049397FB
:103AE0006900A5831377F70F9DBD8547B386E7402F
:103AF00011C76D4601478147E343D6E61307E40942
:103B00003397E9003337E000B3D7D900D98F13F7E3
:103B1000770019C713F7F70091466303D7009107A1
:103B200013975700634C07009A07A583014705BD0B
:103B30001307F00F814725B52E84B5B70547814798
:103B400039BD3707800041117D179356750113D891
:103B50007501B377A70093F6F60F935EF501337600
:103B6000B70026C24AC01378F80F06C622C4130352
:103B7000F00F3E8E3689F684139F3700FD811315B2
:103B80003600B38806416302681093C51500638C44
:103B9000BE106354100D631008106304051EFD1859
:103BA000B307AF40638608029307F00F6388F616E9
:103BB000ED4763C71729130700023307174133176F
:103BC000E500B35715013337E000D98FB307FF4045
:103BD000139757006351071A370400047D147D8C36
:103BE00022850D256D15B317A400634E251B3305E3
:103BF00025411304150013070002018F3397E700D6
:103C00003337E000B3D78700D98F014913F7770026
:103C100019C713F7F70091466303D700910713976D
:103C20005700635E0714930619001307F00F93FE05
:103C300014006386E6169A07A58393F6F60FA60787
:103C4000B240224413D59700DE069397FE01558DAE
:103C5000924402495D8D410182806392080A138774
:103C600016001377E70F631B0714639406226302A1
:103C70000F2071D5B307AF40139757006355072244
:103C8000B307E5410149AE8451B7E30005F0638A0B
:103C9000BE0AE35410FD9307F00F6381F608B707DF
:103CA00000045D8D31B7635E100963010808930756
:103CB000F00F6385F606B70700045D8DED4763C01E
:103CC000171F13070002330717413317E500B357D7
:103CD00015013337E000D98FFA9713975700635CCB
:103CE000070805091307F00F630BE90AB706007E02
:103CF00013D71700FD16858B758FD98F01BF33073A
:103D0000D84063950610630D0F147D176303071ADF
:103D10009307F00F6314F810AE84328E630F0E0613
:103D2000814E9306F00FB707400011BF39C9FD1847
:103D3000B307AF00E38308FA9307F00FE390F6F8B8
:103D4000F1BF63990808138916001377E90F63160A
:103D50000712639B061063030F16E30205EEB30719
:103D6000AF0013975700014963570700370700FC5E
:103D70007D17F98F054913F77700E31C07E813DE79
:103D800037009307F00FE30BF9F893179E00A58314
:103D90009376F90F93FE14005DB593FE140093061D
:103DA000F00F814769BD370700FC7D17F98F13F7C6
:103DB00077003309A940E31E07E4D1B73304AF40CD
:103DC0009317540063C3070CE31C04E0814E814643
:103DD0008147B5B53307D840B5C69307F00FE30E5A
:103DE000F8F2B7070004336FFF00ED4763CDE70C2F
:103DF00093070002998FB317FF003357EF00B337D3
:103E0000F0005D8FB307A7004289C1BD9307F00F93
:103E1000E304F8F0B7070004336FFF00ED4763C217
:103E2000E70893070002998FB317FF003357EF009D
:103E3000B337F000D98FB307F5404289AE8449BB50
:103E4000854769B3630E0F067D17B307AF0042893C
:103E5000E30507E89307F00FE319F8F8328E7DBD0C
:103E6000328E4289AE8431BFE3090FEAE30805EAE6
:103E700045BD0DCDAE8EB287D9B39307F00FE300E9
:103E8000F9F2B307AF008583FDB53304E541AE8495
:103E900081BBE31D0FFCE30505E8AE84BDBD85478E
:103EA00025BD854749BF0149E39707EC814E81470E
:103EB00079B3B307E5414289AE8419BBB28741B3F8
:103EC000328E42897DBD054735BF135775013706D0
:103ED00080009307F6FF1377F70F9305E007B3F61B
:103EE000A7009357F501014563F4E50099C382806B
:103EF00082809307E0097D55E3EBE7FE93055009C7
:103F0000B3E7C60063D7E5001307A7F63395E700CC
:103F10008280130560093307E54033D5E7008280CE
:103F2000411106C622C415CD2A84E92C9307E00965
:103F30003387A7409307600963C0E704A1469377DE
:103F4000F70F63D5A60061153314A400260425805D
:103F5000260413559400B2402244DE075D8D4101D2
:103F600082800144260413559400B24022448147C4
:103F7000DE075D8D410182809307900963DDE700D4
:103F80009307B5019546B317F400898EB337F00057
:103F90003354D4005D8C954763D6A7009307B5FFD3
:103FA0003314F400B70600FCFD16937774003376E3
:103FB000D40085C39377F4009145638CB700110654
:103FC0009317560063D707009307F009758E338760
:103FD000A740131466002580260413559400B240B0
:103FE00022449377F70FDE075D8D410182801357DE
:103FF00075011377F70F41119307170022C426C2EA
:104000001314950006C693F7E70F25809354F50126
:1040100085C793573400130707387604B207520751
:10402000B1831395F401D98FC98FB2402285224400
:104030009244BE854101828005EB39C42285D92294
:10404000A94763C6A7042D47098F93075501335726
:10405000E4003314F4009317C70013079038098F56
:10406000B1831377F77F5DBF01CC13573400B707D7
:104070000800D98FB2077604B1831307F07F79BFA8
:104080001307F07F814759BF0147814741BF13079D
:1040900055FF3317E40001447DBF93D64501939744
:1040A000C50093F6F67FB183138616008E0713576B
:1040B000D5011376E67FFD815D8F9318350035CEEF
:1040C000138806C89307E00F63DD07018147139546
:1040D00097009306F00FDE062581FE05558D4D8D68
:1040E00082806355000B931765000E07B337F0000D
:1040F000D98F93D8D801B3E7170113F7770063017D
:10410000071013F7F70091466303D70091073707AD
:1041100000047D8F75C7130718001306F00F937600
:10412000F70FE305C7FA9A07A58313959700DE06F4
:104130002581FE05558D4D8D8280B367170199EE5F
:1041400085CF95479A07A5831395970093F6F60FA9
:10415000DE062581FE05558D4D8D8280A5DBB707D6
:104160004000139597009306F00FDE0681452581E8
:10417000FE05558D4D8D82808147139597008146B0
:10418000DE062581FE05558D4D8D8280A55763483D
:10419000F804F94737068000B38707417D45598EFB
:1041A0006351F5047957330707411305000233576C
:1041B000E6006388A700938626CAB316D600B3E844
:1041C000D800B3371001D98F13F77700014815FBDA
:1041D000139757008546E34807F48146A5B7814603
:1041E0008DB7938626C83397D8003337E000B316CF
:1041F000D600B3D8F800B367D700B3E7F800E9B743
:10420000C28689B7C167637CF5029307F00F130775
:10421000000263EBA7009717000093876766AA97D1
:1042200088233305A7408280218197170000938758
:104230002765AA97882361473305A7408280B7077F
:104240000001636DF5006181971700009387476354
:10425000AA97882321473305A74082804181971779
:1042600000009387E761AA97882341473305A74059
:104270008280B3C7A5008D8B3307C50081E78D47CA
:1042800063EDC700AA87637EE5089421850785054D
:10429000A38FD7FEE3EBE7FE828093763500AA87F3
:1042A00089CA942185078505A38FD7FE93F6370029
:1042B000C5BF9376C7FF138606FE63F0C70683A3C8
:1042C000050083A2450083AF850003AFC50083AE20
:1042D000050103AE450103A3850183A8C5019385AC
:1042E000450223A0770003A8C5FF23A2570023A4FB
:1042F000F70123A6E70123A8D70123AAC70123AC0E
:10430000670023AE17019387470223AE07FF75B7F7
:1043100090419107910523AEC7FEE3EBD7FEE3E69C
:10432000E7F6828039713EDA2ED232D436D63AD8C8
:1043300042DC46DE9387018122CC804326CA06CE2A
:10434000AA8409C41C4C99E32285FD290C4454100D
:104350002686228536C6EF009013F2406244D2448E
:1043600021618280011126CA4AC806CE22CC4EC6DF
:1043700052C4AA842E8901C51C4D91E3F1219C4CA5
:10438000804499E32685C9219717000093874761E8
:10439000631BF402C0405E24A18BB1C71C48A1C7B7
:1043A000FD59294A1C4483450900FD17B1E91CC485
:1043B00063DD07062286A94526856920FD57630827
:1043C000F502294535A0971700009387675F6314AE
:1043D000F4008044C9B7971700009387675AE31C1D
:1043E000F4FAC0444DBFA2852685192A55D97D55BA
:1043F000F2406244D2444249B249224A0561828075
:104400001CC4050963D70700184C63CAE70063881A
:1044100045011C401387170018C08CA361B7228682
:1044200026850D20E31035F9D9B71C4013871700F6
:1044300018C0294798A371B793870181AA8588433B
:104440006FF05FF2011122CC26CA4AC806CE4EC6D2
:10445000AA842E89328401C51C4D91E3F526971755
:1044600000009387E7536317F406C0401C4C1CC43C
:104470005E24A18BC1C31C48B5CF1C48084093796A
:10448000F90F1379F90F1D8D5C486346F500A2857D
:104490002685692C25E51C440505FD171CC41C4018
:1044A0001387170018C0238037015C486388A70072
:1044B0005E24858B81CBA9476316F900A2852685EA
:1044C000B5240DEDF24062444A85D2444249B249D6
:1044D00005618280971700009387874E6314F4006C
:1044E000804469B79717000093878749E310F4F871
:1044F000C044ADBFA2852685212041D17D59D9B7C1
:1045000041119387018126C2844322C44AC006C652
:104510002A892E8489C49C4C99E3268535269717D1
:1045200000009387E747631BF402C0400317C400F1
:1045300093170701C18393F68700ADEA93F607014D
:1045400095EEA5472320F900136707045AA47D556B
:10455000B2402244924402494101828097170000F0
:10456000938707466314F4008044C9B79717000087
:1045700093870741E31CF4FAC0444DBF918B9DC360
:104580004C5889C9930744046384F5004A85292B54
:10459000232A04025E242322040093F7B7FD5EA4BD
:1045A0001C481CC05E2493E787005EA41C4899EB5E
:1045B0005E241307002093F707286385E700A28590
:1045C0004A8591295E2413F717001DC35C482324F4
:1045D0000400B307F0401CCC1C480145B5FB831711
:1045E000C40013F707082DD793E707045EA485B727
:1045F000898B014791E3584818C4F9BFDE250111A2
:1046000022CC26CA06CE4AC84EC613F78700AA8413
:104610002E8479EBD841634DE000B841634AE00055
:104620000145F2406244D2444249B2490561828068
:1046300058547DD703A904009396370123A00400A2
:1046400063DB060670485E24918B99C75C401D8E23
:104650005C5899C33C401D8E5C540C5081462685A5
:104660008297FD575A24631DF5009440F54763E88F
:10467000D706B70740208507B3D7D700858BA5C3DA
:104680001C48232204001CC09317370163D807007D
:10469000FD576314F5009C4091E368C84C5823A073
:1046A0002401BDDD930744046384F5002685ED2EC7
:1046B000232A0402B5B70C50014685462685029789
:1046C000FD572A86E311F5F89C40B5DF75476385F1
:1046D000E70059476393E70423A0240191B71367C8
:1046E00007045AA47D5535BF83A90501E38A09F261
:1046F00003A905008D8B23A03501330939410147FA
:1047000091E3D84918C4E35D20F11C540C50CA86CB
:104710004E86268582976347A0005E2493E70704B0
:104720005EA4C9B7AA993309A940F1BF9C49A5C3A2
:10473000011122CC06CE2A8411C51C4D81E72EC65C
:104740002122B2459717000093878725639CF500C7
:104750004C408397C5009DC722856244F2400561A5
:104760006FF0DFE997170000938787256394F500C2
:104770000C44C5B79717000093878720E39BF5FC8F
:104780004C44C1BFF240624401450561828001454D
:104790008280411122C406C62A844EA572A5232018
:1047A00005002322050023240500232205062328D3
:1047B0000500232A0500232C050021468145130509
:1047C000C505EFB0FF9D97170000938787B25CD0B7
:1047D000971700009387A7B41CD4971700009387FE
:1047E00087B85CD4971700009387E7BA00D01CD82D
:1047F000B24022444101828097050000938545F331
:1048000091AA411126C2130680069384F5FFB38452
:10481000C4024AC02E8922C406C6938544070D2EC1
:104820002A8401CD2320050023222501310508C457
:10483000138684068145EFB0BF962285B24022449C
:1048400092440249410182801C4DA5E7411106C6F0
:1048500022C497070000938767FA1CD5938741818C
:104860009C432324050423260504232805046314FC
:10487000F50085471CCD2A84352848C022851D288F
:1048800008C42285052848C4484001469145EFF0F8
:104890005FF008440546A545EFF0BFEF48440946E0
:1048A000C945EFF01FEF85471CCCB24022444101BF
:1048B0008280828041119387418126C284434AC00D
:1048C00006C69C4C22C42A8981E72685EFF0DFF7D3
:1048D000938484048044DC40FD1763D607009C4029
:1048E000B9CF8440C5BF0317C40039E7C177850736
:1048F000232204062320040023220400232404008E
:104900005CC423280400232A0400232C040021462D
:1049100081451305C405EFB0BF88232A0402232C68
:10492000040223240404232604042285B2402244E2
:1049300092440249410182801304840671BF91456B
:104940004A85EFF01FEC88C049FDB1472320F900EC
:104950000144E1BF797122D44AD052CC56CA5AC818
:104960005EC606D626D24ECE2A8AAE8A13048504A7
:104970000149054BFD5B09ECB25022544A85925423
:104980000259F249624AD24A424BB24B4561828097
:10499000044483294400FD1963D409000040E1BFA9
:1049A000DE24637BFB008397E40063877701A685A1
:1049B0005285829A3369A90093848406E9BF1971EC
:1049C000A6DAAE848395E500A2DC86DE328463DB62
:1049D0000500DE2423A0060093F7070885E7930768
:1049E00000401DA0300836C6EF007020B246E342FA
:1049F00005FE7247BD67F98F7977BA9793B71700AD
:104A00009CC2F1BF930700041CC0F6506654D654F4
:104A1000014509618280DE25011122CC06CE26CA1D
:104A20004AC8898B2E8489CF930774041CC01CC884
:104A300085475CC8F2406244D244424905618280A5
:104A400074003000AA84EFF09FF7A2452A892685DA
:104A5000012219E98317C40013F7072061FFF19BB6
:104A600093E727005EA4C9B797070000938707D98B
:104A70009CD45E2408C008C893E707085EA4A24738
:104A80005CC8B24781CF8315E4002685EF00D018BB
:104A900011C55E24F19B93E717005EA45E24336981
:104AA000F9002316240179B7DDC183A7C5FF4111A1
:104AB00022C406C626C21384C5FF63D307003E94F2
:104AC000AA84EF00301C9387C1859C4381EF232289
:104AD000040023AE81842244B240268592444101E1
:104AE0006F00701A637EF40014403307D40063969D
:104AF000E7009843DC43369718C05CC0D9BFBA873B
:104B0000D84319C3E37DE4FE94433386D700631F83
:104B100086001040B29694C33386D700E31DC7FACF
:104B200010435843B29694C3D8C375B76375C40095
:104B3000B1479CC04DB71040B306C4006316D70000
:104B400014435843B29614C058C0C0C369B782809A
:104B5000011126CA93843500F19806CE22CC4AC8AA
:104B60004EC6A104B14763F3F404B14463E2B40454
:104B70002A89EF0030119387C18598433A8439E040
:104B8000938701869C4391E781454A85252F23A081
:104B9000A186A6854A853D27FD5963193507B1478A
:104BA0002320F9004A85EF00100E29A0E3D004FC71
:104BB000B1471CC10145F2406244D2444249B24966
:104BC000056182801C40858F63CF0702AD4663F686
:104BD000F6001CC03E9404C031A05C406313870201
:104BE00023AEF1844A85EF00100A1305B400930741
:104BF000440061993307F5405DDF3A94898F1CC00A
:104C00005DBF5CC3C5B72287404095BF1304350024
:104C10007198E30285FCB305A4404A856525E31C31
:104C200035FBB5BF1C46FD171CC663DA0700184EDE
:104C300063C5E700A9476394F5006FF0BF801C428D
:104C40002E851387170018C28CA38280011122CCF5
:104C500026CA4AC84EC652C406CE2A89AE893284B4
:104C6000B304D6007D5A63149400014509A80C20B2
:104C70004E864A85EFF01FFB0504E31645FFF24020
:104C80006244D2444249B249224A05618280357168
:104C900022CD26CB4AC94EC706CF52C556C35AC1EC
:104CA000DEDEE2DCE6DAAA89AE843289368409C522
:104CB0001C4D99E3EFF05FB997170000938747CE3B
:104CC0006398F40C83A44900DE24A18BE5C79C48BB
:104CD000F5C393070002A304F1029307000302D275
:104CE0002305F10222C6930B5002971A0000938A03
:104CF0002ACF054C294B4A841C2099C3639F770D0A
:104D0000B30C2441638E0C00E6864A86A6854E8548
:104D1000EFF0DFF3FD57630FF51C9256E69636D29F
:104D20001C206389071CFD571309140002C802CE1A
:104D30003ECA02CCA309010482D48345090015466A
:104D400056852D2713041900C24751E913F70701AF
:104D500009C713070002A309E10413F7870009C775
:104D60001307B002A309E104834609001307A00258
:104D7000638FE606F2474A8481462546182093054C
:104D80001400130707FD6377E60AB5CA3ECE85A86F
:104D9000971700009387C7C26395F40083A4890026
:104DA00025B7971700009387A7BDE39FF4F083A46E
:104DB000C90019BFA6854E85EFF08FF419D97D552E
:104DC000FA406A44DA444A49BA492A4A9A4A0A4B9A
:104DD000F65B665CD65C0D618280050431BF3305ED
:104DE00055413315AC00C98F3EC82289B9B7324747
:104DF00093064700184336C6634707023ACE182089
:104E00009307E002631DF70418309307A002631BA9
:104E1000F702B2470904138747009C433AC663C1AF
:104E200007023ECA2DA83307E04093E727003ACE99
:104E30003EC8F1B7B387670385462E84BA973DBF56
:104E4000FD57C5B7050402CA81468147254618208B
:104E500093051400130707FD6374E606F9F20C20AE
:104E60000D4617150000130525B8092511CD971714
:104E70000000938767B71D8D93070004B397A700C1
:104E8000424505045D8D2AC80C20194617150000FF
:104E90001305C5B5130914002304B102C12B35C194
:104EA00097B7FFFF9387071695E74247B2471377F7
:104EB000071009CF91073EC69257D2973ED225BD23
:104EC000B387670385462E84BA9751B79D07E19B48
:104ED000A107D5B7780097060000938666D7268687
:104EE0000C084E8597000000E7000000FD572A8A55
:104EF000E314F5FCDE2493F70704E39207EC125564
:104F0000C1B5780097060000938686D426860C08E3
:104F10004E85012AE1BF797156CA9C49BA8A9845E3
:104F200022D426D24ECE52CC06D64AD05AC85EC61D
:104F3000AA892E84B284368A63D3E700BA879CC0DC
:104F40000347340419C385079CC01C4093F707022C
:104F500081C79C4089079CC003290400137969001C
:104F6000631A0900130B9401FD5B5C449840998F10
:104F7000634CF9041C408346340493F70702B336AC
:104F8000D000A5EB13063404D2854E85829AFD57D6
:104F90006303F5041C4011469840998B54448144A6
:104FA0006397C700B384E64063D3040081441C4484
:104FB00018486354F700998FBE94014969047D5BDA
:104FC00063982405014509A885465A86D2854E85F1
:104FD000829A631E75017D55B25022549254025933
:104FE000F249624AD24A424BB24B4561828005097E
:104FF000ADBF3307D40013060003A301C704034762
:10500000540493871600A2978906A381E7049DBFE5
:1050100085462286D2854E85829AE30E65FB050978
:1050200045B7797122D426D24AD04ECE06D652CC7C
:1050300056CA5AC8B689942D930790063289AA8415
:105040002E8413863504638DF60263E2D706930738
:1050500080056386F61863EDD700638E06209307FC
:105060003004638EF60A930A24042301D404C9A0F1
:10507000930730066385F60A93074006E395F6FE2C
:105080001C40084393F6070893054500C5C61C411C
:105090000CC363D807001307D002B307F040A30185
:1050A000E404971600009386E694294765A89307C1
:1050B00000076382F61663E5D7029307E00663896B
:1050C000F6189307F006E390F6FA0C401C4313F829
:1050D0000508138547006307080608C39C4385A895
:1050E00093075007E383F6FE930780076389F61260
:1050F00093073007E399F6F61C43D0418145938628
:10510000470014C383AA070056858D2601C53305C1
:10511000554148C05C401CC8A301040461A81C435D
:10512000930A2404938647009C4314C32301F40488
:105130008547D5B793F607041C410CC3B9DAC207FB
:10514000C18781BF93F5050408C3C9D99E231307FE
:10515000F0066387E60E971600009386A689294716
:10516000A30104044C400CC463C5050008406D99BC
:1051700008C099E3B28A89CDB28AB3F5E702FD1A75
:10518000B6958C212380BA00B3D5E70263F0E70C13
:10519000A147631EF7001C40858B91CB58401C48EB
:1051A00063C7E70093070003A38FFAFEFD1A3306D7
:1051B000564110C84E87CA867000A2852685EFF03A
:1051C0009FD57D5A631D450B7D55B2502254925494
:1051D0000259F249624AD24A424B45618280A38217
:1051E000D504971600009386E6800C40084313F818
:1051F00005081C411105630D080208C313F71500CB
:1052000001C793E505020CC04147B9FB0C4093F57B
:10521000F5FD0CC0B1B79C4193E707029CC1930711
:105220008007A302F404970600009386E67D75BF0D
:1052300013F8050408C3E30308FCC207C1837DBF5C
:10524000970600009386067B214719BFAE8735B7C6
:1052500094411C43CC4913F80608138547006306A4
:10526000080008C39C438CC339A008C393F6060406
:105270009C43F5DA8EA323280400B28A25BF144884
:105280005686CA8526858299E30045F51C40898BA0
:105290008DE7B2474844E35AF5F23E853DB785466F
:1052A0005686CA8526858299E30065F3050A5C4423
:1052B0003247998FE345FAFEE9BF014A930A940108
:1052C0007D5BF5B7411122C42A842E8523A201AE4D
:1052D00006C6EFC05FD5FD576317F500938741AE53
:1052E0009C4391C31CC0B2402244410182804111C1
:1052F00022C42E848395E50006C679226349050001
:105300007C48AA977CC8B2402244410182805E2436
:105310007D777D17F98F5EA4FDB7DE25011122CCC4
:1053200026CA4AC84EC606CE93F70710AA842E8412
:105330003289B68991C78395E500894601460922DD
:105340005E247D777D17F98F5EA48315E4006244A7
:10535000F240CE864A86B24942492685D24405614A
:1053600025A8411122C42E848395E50006C6C928CC
:10537000FD575A24631AF500FD77FD17F98F5EA4D7
:10538000B2402244410182808567D98F5EA468C8FB
:10539000C5BF8395E50005A8411122C42A842E8546
:1053A000B285368623A201AE06C6EFC0FFC3FD5705
:1053B0006317F500938741AE9C4391C31CC0B24074
:1053C000224441018280411122C42A842E8523A2D5
:1053D00001AE06C6C520FD576317F500938741AEA1
:1053E0009C4391C31CC0B2402244410182804111C0
:1053F00022C42A842E85B28523A201AE06C6C92006
:10540000FD576317F500938741AE9C4391C31CC0C1
:10541000B240224441018280411122C42A842E8557
:1054200023A201AE06C65D20FD576317F5009387E2
:1054300041AE9C4391C31CC0B240224441018280D2
:10544000411122C42A842E85B285368623A201AE5C
:1054500006C65920FD576317F500938741AE9C435C
:1054600091C31CC0B24022444101828093F5F50FE4
:105470002A966314C500014582801C21E38EB7FE85
:105480000505C5BF82808280411122C42A842E85F1
:10549000B285368623A201AE06C6A920FD57631742
:1054A000F500938741AE9C4391C31CC0B240224497
:1054B000410182809307800523A2F1AE7D55828051
:1054C0009307800523A2F1AE7D5582809307800566
:1054D00023A2F1AE014582809307800523A2F1AE9D
:1054E0007D5582809307800523A2F1AE7D55828091
:1054F00053797374656D436C6B3A25640D0A000033
:105500004368697049443A253038780D0A00000034
:1055100043616C696272617474696F6E5F56616C2D
:10552000203A2025640A000025640A0025640D0A3B
:1055300000000000CDCC4C3D6666663F0000F043A5
:105540009A9999999999A93FCDCCCCCCCCCCEC3FE8
:10555000696E2074696D312069727120000000004D
:10556000010AA03B00000000000000000000E03F36
:10557000000000000000344003D25E3CC10DDC3B63
:105580001D130F130213F412E612D712C812B91228
:10559000AA129A128A127A126A12591248123712F1
:1055A000251213120112EE11DB11C811B511A11150
:1055B0008D11791164114F113A1125110F11F91044
:1055C000E310CC10B5109E1087106F1057103F10CD
:1055D00026100D10F40FDB0FC20FA80F8E0F740FE3
:1055E000590F3F0F240F090FED0ED20EB60E9A0E73
:1055F0007E0E620E460E290E0C0EF00DD30DB60D6A
:10560000980D7B0D5E0D400D220D050DE70CC90CAC
:10561000AB0C8D0C6F0C510C330C150CF70BD90B1C
:10562000BB0B9C0B7E0B600B420B240B060BE80A9A
:10563000CA0AAD0A8F0A710A540A360A190AFC0905
:10564000DF09C209A50988096C094F09330917093F
:10565000FB08DF08C308A8088D08720857083C0833
:1056600021080708ED07D307B907A00786076D07CC
:1056700054073C0723070B07F306DB06C406AD06F9
:1056800096067F06680652063C0626061006FB05AF
:10569000E605D105BC05A70593057F056B055805F3
:1056A000450532051F050C05FA04E804D604C404B8
:1056B000B304A10490047F046F045F044E043E040D
:1056C0002F041F0410040104F203E303D503C703EE
:1056D000B903AB039D0390038203750368035C0366
:1056E0004F03430336032A031F0313030703FC027C
:1056F000F102E602DB02D102C602BC02B202A7023C
:105700009E0294028A02810277026E0265025C02A6
:1057100054024B0242023A0232022A0222021A02C6
:1057200012020B020302FC01F401ED01E601DF01AC
:10573000D801D201CB01C401BE01B801B101AB0156
:10574000A5019F01990194018E01880183017D01CA
:10575000780173016E01690163015E015A0155010F
:10576000500100000000803F00007A440000C84261
:105770000000304100007041CDCC4C3F16D3FFFFFC
:1057800008D2FFFF08D2FFFF06D2FFFF0ED2FFFFB5
:105790000ED2FFFFD4D1FFFF06D2FFFF0ED2FFFFD4
:1057A000D4D1FFFF0ED2FFFF06D2FFFF02D3FFFFCF
:1057B00002D3FFFF02D3FFFFD4D1FFFFE8DEFFFFDC
:1057C0000EDEFFFFE2DEFFFF16DEFFFFE2DEFFFF81
:1057D000DCDDFFFFE2DEFFFF16DEFFFF0EDEFFFF78
:1057E0000EDEFFFFDCDDFFFF16DEFFFF1CDEFFFF2E
:1057F0001CDEFFFF1CDEFFFFDCDDFFFFCEDDFFFF59
:10580000CEDDFFFFA2DEFFFF7EDFFFFFA2DEFFFF98
:105810009CDDFFFFA2DEFFFF7EDFFFFFCEDDFFFF8F
:10582000CEDDFFFF9CDDFFFF7EDFFFFFDCDDFFFF46
:10583000DCDDFFFFDCDDFFFF9CDDFFFFF6E1FFFFAE
:1058400044E1FFFF44E1FFFF42E1FFFF48E1FFFFCA
:1058500048E1FFFF18E1FFFF42E1FFFF48E1FFFFE2
:1058600018E1FFFF48E1FFFF42E1FFFFE4E1FFFF36
:10587000E4E1FFFFE4E1FFFF18E1FFFF00010202A6
:1058800003030303040404040404040405050505D8
:1058900005050505050505050505050506060606B4
:1058A0000606060606060606060606060606060698
:1058B0000606060606060606060606060707070784
:1058C0000707070707070707070707070707070768
:1058D0000707070707070707070707070707070758
:1058E0000707070707070707070707070707070748
:1058F0000707070707070707070707070808080834
:105900000808080808080808080808080808080817
:105910000808080808080808080808080808080807
:1059200008080808080808080808080808080808F7
:1059300008080808080808080808080808080808E7
:1059400008080808080808080808080808080808D7
:1059500008080808080808080808080808080808C7
:1059600008080808080808080808080808080808B7
:1059700008080808080808080808080800000000C7
:105980000000000000000000000000000000000017
:105990000000000000000000000000000000000007
:1059A00000000000000000000000000000000000F7
:1059B00000000000000000000000000000000000E7
:1059C00000000000000000000000000000000000D7
:1059D000000000000000000000000000232D302B1C
:1059E00020000000686C4C00656667454647000073
:1059F0003031323334353637383941424344454605
:105A000000000000303132333435363738396162C6
:085A10006364656600000000FC
:105A18000000000000000000010203040607080956
:105A2800000000000102030401020304060708093C
:105A380000000000000000000000000000E8038CE7
:105A4800051400A406DC05A00564008C050A000105
:105A580000140014004600320028000A003C001020
:105A68000E000000534C1111111111111101000108
:105A78000016000000000000030000008025000060
:105A8800000000000000000000000000000000000E
:105A98000000000004000000802500000000000055
:105AA80000000000000000000000000000000000EE
:105AB8009C590000BC5900007C59000000000000FF
:105AC80000000000000000000000000000000000CE
:105AD80000000000000000000000000000000000BE
:105AE80000000000000000000000000000000000AE
:105AF800000000000000000000000000000000009E
:105B0800000000000000000000000000000000008D
:105B1800006CDC0202040608E80300200000403F95
:085B28009C0000209C000020FD
:00000001FF
